:100000000AC018951895189518951895189518956B
:100010001895189518958FE181BD87E181BD8FED09
:100020008DBFC0ECE8EB4E2EDD275D2EEEE7F0E055
:10003000A0E6B0E088278D933197E9F78FE289B980
:1000400088E18AB966248FEF87BB18D1E8EFF6E024
:100050000FD214D213D2E1E0F0E0A0E698E32CD363
:10006000ECE0F7E005D2A0E6FDD108D207D2E9E343
:10007000F0E0A8E991E020D3EEE1F7E0F9D1A8EAB9
:10008000B0E0E8E9F0E069D2EBD1EEE2F7E0F0D1E0
:10009000F5D1F4D1F3D1E4E3F7E0EAD1EFD1EED139
:1000A000EAE3F7E0E5D1EAD1ECE4F7E0E1D1E6D12B
:1000B000ECE5F7E0DDD1E2D1E4E6F7E0D9D1DED13D
:1000C000A6EA52D1A6EA0D911C91083E5DEF1507F4
:1000D00009F006C0A5EA8C918F5F8C93A6EA07D23F
:1000E0000091A5000C3009F001C01CC05F9BE8CF57
:1000F00033E098D1A8EAB0E07AD2A9E90C93BED156
:1001000000919900013009F002C0D6D00BC0023036
:1001100009F002C0E3D006C0033009F002C002C0FB
:1001200001C099CFABD0ECE6F7E0A2D1A7D10CE3A8
:1001300010E0A8E94D91552728D1AFE94D935C9384
:10014000AFE90D911C9144E150E01AD1AFE90D9354
:100150001C93A0E6B8D2A3EA8C9381E08093A4001C
:100160004091A3000091A400041710F009F071C0A1
:100170008091A400E0E6F0E001E00A93AAE969D2E8
:10018000EAE9F0E0AAE9BBD1AAE98C91A1EA8C9353
:10019000AAE9E6E7F7E09DD209F002C062D053C0B9
:1001A0000091A1000F3381E008F480E08F9300916B
:1001B000A1000B3581E010F009F080E09F918923C8
:1001C000882309F402C060D014C00091A1000C3251
:1001D00081E008F480E08F930091A1000A3381E070
:1001E00010F009F080E09F918923882309F401C071
:1001F00057D088E090E0ACE98D939C9391E0A2EA1F
:100200005CD1ACE9B7D0A2EA0C9107FB0EF0F6CFB7
:10021000ACE9B0D091E0A2EA50D1C09AA2EA0C9128
:1002200007FB0EF002C018D001C01BD0C09814D03C
:10023000ACE9A0D0ACE90D911C91003050E015075D
:1002400009F0E8CF0ED0A4EA8C918F5F8C9309F06F
:1002500087CF83CFF894FFCFAFE98D919C911ED1CA
:100260000895AFE98D919C9119D1AFE98D919C9141
:1002700015D1AFE98D919C9111D108958BE101D1F8
:10028000E8E7F7E0F5D00895A1EA8C918F538C93BD
:10029000EEE3F3E0A1EA8C919927A2EA25D1089533
:1002A000A1EA8C918C528C93EAE5F3E0A1EA8C915F
:1002B0009927A2EA19D10895ECE7F7E0D9D0DED06A
:1002C000A0E637E3B1D0DAD0A0E6CCD0D7D0E1E0D9
:1002D000F0E0A0E698E37BE7E1D10895ECE9F7E0F0
:1002E000C7D033E09FD0A8EAB0E081D1A8E90C9351
:1002F00000919800053081E008F480E08F93009130
:100300009800043181E010F009F080E09F9189238A
:10031000882309F407C0E9E3F0E0A8E991E07BE76E
:10032000AFD101C0DBCFAAD0A8EAB0E0E8E9F0E0A5
:1003300014D196D0EEE2F7E09BD0A0D0089573657B
:100340000617150B031D091F07180A1B04050819BA
:10035000120D0F020E1E0C1614134C736A2D203052
:10036000383C3E3F2F272321ED91FC913196FC93A1
:10037000EE930895ED91FC913197FC93EE930895DF
:1003800008D03DD000FC10D0089503D01ED001F855
:10039000F9CF0024E89457FF02C009D0689400F810
:1003A0000BD010F80124089502D009D0089550957B
:1003B00040954F5F5F4F0895E89417FF08950095AB
:1003C00010950F5F1F4F68940895352F242FE894E0
:1003D000452B11F468940895512F402F00271127C1
:1003E00080E1440F551F001F111F021B130B4160BA
:1003F00018F4020F131F4E7F8A9599F70895752FF1
:10040000642F55274427FF93F1E1889405C010F429
:10041000460F571F5695479517950795FA95B9F7C3
:10042000FF910895A8EAB0E017D08D3049F08830E8
:1004300079F03323C9F38D933A9563FE22D0F4CF3C
:1004400063FC03C01ED08AE01CD088278C930895DB
:1004500018D011973395E8CF5F9BFECF8CB10895EC
:10046000A8EAB0E08D91882311F00BD0FBCF08955E
:100470002CD0802D11F005D0FBCF08958DE001D058
:100480008AE05D9BFECF8CB908953197F1F708950E
:10049000689462F80895E89462F80895EF93FF93E2
:1004A000EE27E82BE92B31F0E3E3F7E03197F1F7A2
:1004B0000197D1F7FF91EF910895903029F08C9139
:1004C000880F9A95E9F78C930895C8953196002086
:1004D000089581E003C082E001C084E0C8950D92D8
:1004E00031968A95D9F70895E80FF91FF2CF82E087
:1004F00001C084E099279D938A95E9F70895819139
:1005000004D08D938823D9F70895813618F08B375E
:1005100008F48F7D0895040F151F261F371F0895B7
:10052000000F111F221F331F08950095109520956D
:1005300030950F5F1F4F2F4F3F4F0895019110814E
:100540000EC001911191219130810BC00191108158
:1005500017FF05C03FEF2FEF04C0008111272227AE
:10056000332737FF03C0E1DF8DE28D93CF93DF9315
:10057000CF92DF92EF92AA24BB24CC24DD24EE2478
:1005800040E2CAE0DD2755E093E38881890F87FDCB
:100590009F7083FD907F891B89935A95A9F7C0DFCF
:1005A000AA1CBB1CCC1CDD1CEE1C4A9551F7E89420
:1005B000EFE0FF2782910ED0EB30E0F71EF0689459
:1005C0008A2D0CD088278D93EF90DF90CF90DF910C
:1005D000CF910895982F829501D0892F8F70805DDB
:1005E00026F0803309F4089568948D9308950027C8
:1005F0001127222733271DD08A3328F4803318F09F
:1006000005D015D0F9CF0EF490CF089580538F9375
:10061000402F512F622F732F83DF82DF7CDF80DF3B
:100620008F919927080F191F291F391F08958D9140
:100630000895E894FCDF8032E9F38B32D9F38930F6
:10064000C9F38D3211F46894F2CF089588278D9301
:10065000089509919191992351F08A95D9F731978D
:1006600081918D930A9519F08823D1F70895EECFE3
:10067000E199FECFEEBB3196089591E001C092E082
:100680007B3751F47FB7F894F3DF8D918DBBE29AFD
:10069000E19A9A95C9F77FBF77270895E9DF8D9191
:1006A0007B3729F48DBBE29AE19A8823B9F7772743
:1006B000089591E001C092E0DBDFE09A8DB38D9365
:1006C0009A95D1F708958FEF83959D919923E1F73E
:1006D0000895689401C0E894AF93BF938D9116F08C
:1006E000919102C0F2DE902D891718F011F4882341
:1006F000A9F7BF91AF910895564133544F204265F9
:1007000061636F6E204B657965720000437572728C
:10071000656E74206D6573736167653A200043757B
:100720007272656E742053706565643A20002057BC
:10073000504D00004D656E753A00312E20436861C2
:100740006E6765204D65737361676500322E2043C7
:1007500068616E676520537065656400332E2045BF
:100760007869740028312D33293A200052756E6E55
:10077000696E6720210020005B324A004E657720B9
:100780004D65737361676520283630206368617238
:10079000732E206D61782E293A2000004E65772057
:1007A0005370656564202835202D20323020575045
:0607B0004D293A20000073
:00000001FF
